:030000000219FDE5
:03000B000200A848
:03002B000201854A
:03005B0002033667
:0300730002032362
:1000800002030406080C10182030406080040608A3
:100090000C10182030406080A0C00003070F1F051F
:1000A000050D050305030302C2AF306308C2638573
:1000B000798AD2AF32C0D0C0E0206221E525601637
:1000C000E473E525F4C3334009758A00D263F579FA
:1000D00001D4F58AD262D0E0D0D0D2AF32C3E526C7
:1000E000334009758A00D263F57901EEF58AC26260
:1000F000E526F4602F30682520720DD0E0D0D0C204
:1001000095C293C297D2AF32C295C293C297206F65
:100110000C2065097412D5E0FDE57B4290D0E0D05B
:10012000D0D2AF32758A00D263757900C28DD262A7
:10013000211D01C2306805206502D29501C23068D8
:1001400005206502D29701C2306805206502D2936E
:1001500001C2C29430680A2065077412D5E0FDD24E
:100160009501C2C29630680A2065077412D5E0FD79
:10017000D29701C2C29230680A2065077412D5E096
:10018000FDD29301C2C2AFC2AD53E6EFC0D0C0E012
:10019000D2D3D2AFE57A6009E57760057577004183
:1001A000D0757701C2CEE52A600720744F152A2149
:1001B000FC7800790020742EE580307E01F430E573
:1001C0000278FF53DACF207E0343DA20307E0343E8
:1001D000DA10C2D8C271E580307E01F430E50279D0
:1001E000FFC3E89970CB306103752A18207403753A
:1001F0002A18885CD270E86003755F0020740DE5F2
:100200002B6004152B410C43DA01C2D82070024147
:100210007FA85C206102C270207431C3E894F04072
:100220000374F0F8E8C4540F28F87984B703024146
:100230004CC313C3138721200802C313200A06C32B
:10024000C898F8414C28F8500374FFF8C3E8956546
:100250005003E565F88822E52D54066022206B1FC7
:10026000E536C333C333F8E564C313C313F9C39549
:100270002240028922E82522F52250037522FF85BB
:100280002224A824C3E52495614002A8618825E5BD
:1002900066700241C3C3E8AA669A5003E8FAE4F91B
:1002A000EAC333FBE568F45B29400D2567F8E56791
:1002B00060021567400B41C30AC3E5679A50020507
:1002C0006778FF8826C26FC3E52694F84002D26F94
:1002D00020CF0AD0E0D0D043E610D2AD32C2CF0555
:1002E0003AE57A6009E578600575780061197578F6
:1002F000017801E52A6005307402152AC3E55C9493
:10030000014005755F006119756000756900E55F62
:100310002401F55F5003755FFFD0E0D0D043E610B5
:10032000D2AD32C2AF53E67F7592FA7593FFC260C9
:10033000759104D2AF32C2AF53E6EFC2ADC0D0C0A8
:10034000E0C0F0D2D3D2AFA8FBA9FCE57A6007C326
:10035000E913F9E813F8C2D830710261A853DACF73
:10036000207E0343DA10307E0343DA20D271E58029
:10037000307E01F420E502617F88278928A1D553CA
:10038000DACF207E0343DA20307E0343DA10C2D86E
:10039000C271307402A1C17800E580307E01F43072
:1003A000E502A1C1885CA1A953DACF207E0343DA1C
:1003B00020307E0343DA10C271206102818153DA5A
:1003C000CF207E0343DA10307E0343DA20C2D8D236
:1003D0007188578958C3E89555F8E99556F97B0017
:1003E0007E087A00C3E8948CE994005005755B00A0
:1003F0008173882178A2E6A8216055C3E894C8E9F2
:1004000094005008E4D2E4FB7A0A814EC3E8946871
:10041000E994015008E4D2E3FB7A0F814EC3E894DB
:10042000D0E994025008E4D2E2FB7A1E814EC3E880
:1004300094A0E994055008E4D2E1FB7A3C814EC3D4
:10044000E89498E994085008E4D2E0FB7A787E00BA
:10045000C3E89559FCE9955AFD30E70AECF424010C
:10046000FCEDF43400FD755B00C3EC9AED9E500387
:0F047000755B018859895A85575585585678020A
:10047F00A1A9C3E89527F8E99528F9307C02A18D49
:10048F00307B02A18D307A02A18620750281A4E90A
:10049F00FDE8FC81C3E9C313F9E813F8307902A131
:1004AF0086E9C313F9E813F8307802A186E9C3137C
:1004BF00FDE813FC20612CC3EC941CED9402400268
:1004CF0081DAED701EC3EC94C850180529E5297028
:1004DF00021529C3E529940A5002A1C1755C00D207
:1004EF0070A1C1E529600215297888E6F97400200A
:1004FF007F087896B90302789EE624FAFEE434006A
:10050F00FFC3EC9EFCED9FFD9208B90310A20850AB
:10051F0007207609D276A12C307602C276A2085037
:10052F0016B9030DECF42401FCEDF43400FD0205C3
:10053F004678007900A18DB90315EC33FCED33FD3E
:10054F00C3EC940AFCED9400FD50047C007D00C3C5
:10055F00EC94FFED9400400678FF7900A18DEC85B7
:10056F0072F0A4C5F0A2F733F8790040030205A991
:10057F0078FF79000205A9E9C313F9E813F8307C75
:10058F000EE9600278FFC3E81338F8E43400F9C3CA
:10059F00E894FFE99400400278FF885CD2702061F4
:1005AF0002A1C1741FF4552F4BF52FC274EB7002CB
:1005BF00D274752A18307403752A0A306102A1D5D6
:1005CF0020740353DAFE207403752B06D0F0D0E0AD
:1005DF00D0D0D2AD43E6103279010206057903027D
:1005EF000605790A020605791E02060579640206D8
:1005FF000579C80206057817E4D5E0FDD8FAD9F6D3
:10060F00227A147B7802062C7A107B8C02062C7AC5
:10061F000D7BB402062C7A0B7BC802062CE573D532
:10062F00E001227902E4C296D5E0FDD297D5E0FD34
:10063F00C297D5E0FDD296D5E0FDE920E002D29534
:10064F0030E002D293E573D5E0FDE920E002C295D8
:10065F0030E002C2937496D5E0FDD9C9EAF8D5E02F
:10066F00FDD8FBDBB8C29622C37C007D0075F0007D
:10067F0005F0EA33FAEB33FB50F6EB13FBEA13FA10
:10068F00C3E9FFE8FEE89AF8E99BF95004EFF9EEA9
:10069F00F8B3EC33FCED33FDD5F0DFEDF9ECF822D8
:1006AF00E889F08A20D2D4F8A9F07B0030F70B7BD1
:1006BF00FFF42401F8E9F43400F9E88520F0A4AD43
:1006CF00F0F8E98520F0A4AFF0FEED2EF974003FAD
:1006DF00FA7C04C3EA13FAE913F9E813F8DCF48B94
:1006EF00F030F70AE8F42401F8E9F43400F9E88966
:1006FF00F0C2D4F8A9F02222C3E54113F9E5401363
:10070F00F8C3E54498F8E54599F9500CC3E894808F
:10071F00E994FF401602073EC3E8947FE994005026
:10072F000302073E787F790002073E788079FF88C1
:10073F0049894A22E5492546F8E54A3547F9854A68
:10074F0020E4300701F43548FA30E709C3EA94F0A2
:10075F00401502077CC3EA940F500302077C78FF11
:10076F0079FF7A0F02077C780079007AF0C3E524CD
:10077F009561500AC374019524500B02079AE54AFC
:10078F0020E70E02079AE54A30E706884689478A2E
:10079F00482278A5E6FAC3E54933F8E54A33F9D19B
:1007AF00AFE930E70BC3E89480E994FF4013E1D43D
:1007BF00C3E8947FE994005002E1D4787F7900E197
:1007CF00D4788079FFE820E715C3E52398F840092E
:1007DF00C3E8940140030207FB78010207FBE8F42A
:1007EF0024012523F840030207FB78FF884B22786A
:1007FF00A6E6FAA847A9481206AFE930E70CC3E806
:10080F009401E994FF4016020830C3E894FFE9947D
:10081F0000500302083078FF790002083078017920
:10082F00FFE920E715C3E54B98F84009C3E89401A9
:10083F0040030208577801020857E8F42401254BBA
:10084F00F8400302085778FF88242278FF20692890
:10085F0079A1E76023E541601F74FF8541F084852E
:0E086F0039F0306A0375F005A4F8C5F0600298
:10087D0078FFC3E895645002A864886322C3E540FD
:10088D0094C8E5419400E563500314019B04600294
:10089D00F563220208A32275E890227883E6FF30E3
:1008AD00EDF9A8BDA9BE0570C3E570940840527559
:1008BD007000E9FA79A0E76044EA7007E571601B02
:1008CD000208DCC3E895716010E5715006600C14E8
:1008DD000208E80460F90208E8E571F571C3947245
:1008ED00401B7561C0C394044013756180C39404AB
:1008FD00400B756140C39404400375610075BB08DE
:10090D0022E561F460020561E570B4070375BB1063
:10091D0022743279A787F0A4C5F0A2F733F8C3E8A3
:10092D0095614002A86188228824882588268864DC
:10093D00227540007541F022C2AF75C820A8CCA920
:10094D00CDAA3A30CF010A75C824D2AFC3EA13FA43
:10095D00E913F9E813F8AB3BAC3C883B893CC3E8A1
:10096D009BF8E99C20690A547FF9306602416421A5
:10097D00BEAD3D8A3DF9EA9D547FFA600678FF7958
:10098D00FF21A3AE3EAF3F8B3E8C3FA83BA93CC39E
:10099D00E89EF8E99FF9C3E54113FBE54013FAE83A
:1009AD002AF540E93BF54150067540FF7541FF4181
:1009BD000BAA40AB41AC40AD417E047F02C3EB942A
:1009CD0004400D1E1FC3EB94084005206A021E1F34
:1009DD00C3ED13FDEC13FCDEF7C3EA9CFAEB9DFBB4
:1009ED00EF6009C3E913F9E813F8DFF7EA28FAEB2A
:1009FD0039FB8A408B4150067BFF8B408B41C3EB0B
:100A0D0094025002D2663069047F0341367892E633
:100A1D00FFC3E537948240110FC3E53794A0400121
:100A2D000FC3EF940640027F057E02E541C4540FCB
:100A3D00F9E541C454F0F8E540C4540F28F8C3E873
:100A4D009EFAE99400FB4009C3EA9402EB9400502E
:100A5D00047A02E4FB41B0AA40AB41EBC4FEEAC408
:100A6D00540F4EFCC3EA9CFAEB9400FBC3E813C38E
:100A7D0013F8EA28FAEB3400FB8A408B41C3EB9460
:100A8D00024002C2667802EBC4FE7B00EAC4540F3A
:100A9D004EFAC3EA98FA4005C3940250027A0278DE
:100AAD0092E6FF30600241B0855192855293D2603B
:100ABD0043E680C3E49AF8E49BF9C3E833F8E933DD
:100ACD00F93066026143E8FAE9FBD3E913FDE81357
:100ADD00FC88518952C3EF94036038EF20E00DE894
:100AED002CF8E93DF9ECFAEDFB020B0CE828F8E9DE
:100AFD0039F9C3E82402F8E93400F97AFE7BFFC323
:100B0D00EF9403400E8A538B54884D894E8C4F8D34
:100B1D00506177885389548A4D8B4E8C4F8D503050
:100B2D0069127553F07554FF754FF07550FF75517F
:100B3D00F07552FF6177E8FAD3E813FC8851C3EFE3
:100B4D0094036020EF20E007E82CF8ECFA6163E8ED
:100B5D00282402F87AFEC3EF940340088A53884D87
:100B6D008C4F617788538A4D8C4FE568C3335002A3
:100B7D00646BF5683060026181753402D26043E6C2
:100B8D0080E52D5406602DA840A941C3E913F9E86D
:100B9D0013F8306904E92440F9C2AF53E67F75912B
:100BAD0000C3E498F594E499F595759104D26043EA
:100BBD00E680D2AF22D264754300752000306C03FD
:100BCD00752040020BE1D264754300752040306CF6
:100BDD000375200078017901206620E52D5406600B
:100BED0002C2647914E541C313700104F8C394146F
:100BFD0040027814306904781B791BC3E833F8C3BD
:100C0D00E933F9206010E543600C306903D53404F5
:100C1D00D26D819771890543E59B5440B5200281C2
:100C2D008130690908C3E899400118811020640AD0
:100C3D0008C3E899400261E18110C264C2AF53E676
:100C4D007F7591003066127594007595F07591045D
:100C5D00D26043E680D2AF61E1E5417EFFC3334010
:0D0C6D0009C3334005C3334001FEC3E49EBC
:100C7A00759400F595815AC3E5339401500261E1F8
:100C8A0030640261E1D80281958110C26DC2AF530E
:100C9A00E67F759100855394855495759104854D29
:100CAA0092854E93D26043E680D2AFE52D5406601A
:100CBA0008206A020533020CD3306D0D206C0A201D
:100CCA006407158115810215A8227800306402781C
:100CDA0001E53775F007A4F9E5F028F5F0E9A2F087
:100CEA0013A2F113A2F213F537C3947850037537A0
:100CFA0078C3E53795384008D265C295C293C29742
:100D0A00306002A10A854F92855093D26043E680F3
:100D1A0022207D16C2AF754202C296D29430620278
:100D2A00D293D2AF759F11020F0BC2AF754202C2A6
:100D3A0096D292306202D295D2AF759F11020F0BF2
:100D4A00307243207D20C2AF754203900163757BE8
:100D5A0040C293C292306204D297A168D296D2AFAF
:100D6A00759F13020F0BC2AF754203900163757B27
:100D7A0040C295C294306204D297A188D296D2AF6B
:100D8A00759F10020F0B207D17C2AF7542039001A9
:100D9A003EC293306202D297D2AF759F13020F0BF5
:100DAA00C2AF75420390013EC295306202D297D219
:100DBA00AF759F10020F0B207D16C2AF754204C299
:100DCA0094D292306202D297D2AF759F10020F0B63
:100DDA00C2AF754204C292D294306202D297D2AFA5
:100DEA00759F13020F0B307243207D20C2AF7542EC
:100DFA0005900152757B10C297C296306204D29553
:100E0A00C10ED294D2AF759F11020F0BC2AF7542B9
:100E1A0005900174757B04C297C296306204D2931E
:100E2A00C12ED292D2AF759F11020F0B207D17C22D
:100E3A00AF754205900134C297306202D295D2AFA3
:100E4A00759F11020F0BC2AF754205900148C297F8
:100E5A003062EBD293D2AF759F11020F0B207D1631
:100E6A00C2AF754206C292D296306202D295D2AF12
:100E7A00759F13020F0BC2AF754206C294D2963009
:100E8A006202D293D2AF759F10020F0B30724420C8
:100E9A007D20C2AF754201900174757B04C295C270
:100EAA0094306204D293C1B4D292D2AF759F100229
:100EBA000F0BC2AF754201900152757B10C293C2EB
:100ECA0092306205D295020ED5D294D2AF759F1395
:100EDA00020F0B207D17C2AF754201900148C295DF
:100EEA00306202D293D2AF759F10020F0BC2AF7558
:100EFA004201900134C293306202D295D2AF759FFB
:100F0A0013C26522900132757B00C295C293C297C3
:100F1A00C294C292C296C26222788076FF0876FF95
:100F2A000876FF0876FF08760308760408760A082A
:100F3A007603087601087601788C76010876FF0830
:100F4A0076FF0876FF0876FF0876FF0876030876AC
:100F5A00FF0876FF0876FF0876250876D00876FA25
:100F6A000876FA0876040876FF08760108760008FB
:100F7A00767A0876FF087601087601087600087600
:100F8A0003087600227887E6FFC272BF0302D27294
:100F9A007888E6C394036008C27DE630E102D27D18
:100FAA00C27E7889E630E102D27EC3EF94026008FD
:100FBA00758E01D273020FC7758E00C273227880B4
:100FCA00E6149000809378A5F67881E61490008064
:100FDA009378A6F67886E61490008D9378A7F6782B
:100FEA0086E6F539C394025003753902789CE67592
:100FFA0038FFB402037538A0B4030375388278A3A6
:10100A00E61490009A93F566120F0E22227896E65D
:10101A00FA7897E6FB7888E6B40305C3EB940EFBEF
:10102A00307F047A007BFFC3EB9AFCC394825002A0
:10103A007C827572000572EC8572F0A4C3E5F094A7
:10104A007D40F222D27F11171205F61205F67A00B8
:10105A007B007C101205ECE55C2AFA74003BFBDC91
:0F106A00F37C04C3EB13FBEA13FADCF7FEC27F3F
:10107900111722757C00757D00E5EF20E6037520C8
:10108900000520903FFFE520146006901FFF1460C3
:10109900009304600375EF1653D9BF7581C043FFF0
:1010A900801205E775EF0643B203E5B3240220E792
:1010B9000DF521E5E320E0068521B343E301120F95
:1010C9000E7580FF75A40075F1B275D4DF759001B6
:1010D90075A5FC75F2FE75D50175A60175E241127B
:1010E9000F0EE4F8F6D8FD756801120F23121602E7
:1010F90078988673753001C2AF1206001206101275
:1011090005F61206171205F612061E1205F6121733
:101119002B1206001206001205FBC2AF757C007582
:101129007D0078FA79FA308507D9FBD8F7021C00D7
:10113900120F8F120FC81116111778988673120F94
:101149000E75A90075B680757A00758810758902C3
:1011590075C82475910475D84075A82275B80275AB
:10116900E690759B80759D0075D10E75BCC075BBE9
:101179000875BA1175E8801205E7D2AF1208A07593
:10118900360053DACF207E0343DA20307E0343DA78
:101199001043DA01C2D8C271120600D2617B037A08
:1011A9000CE55B70077A0CDB030211231205F620AC
:1011B9007003021123C270E55CC3940240E1E52F7C
:1011C900541F855E5DF55EB55DD5DAD5C26153DA2A
:1011D900CF207E0343DA20307E0343DA10C2D8C21F
:1011E9007178A2E67008D274E52F54E0F52FC27524
:1011F9007529001205FB307409C3E529940A4002D8
:10120900D2751205EC78023074027800C3E55C9857
:1012190040F0C2AF120610120610120610D2AF1219
:101229000600754C007888E6B4030261231205ECC8
:10123900788CE6C394015003021323E530C394016B
:101249005003021323757CA5757DF1207435C3E520
:101259005C94FF5003021323C2AF120625D2AF12CA
:1012690005FBC3E55C940150EFC2AF1206101205ED
:10127900F1120610D2AF1205FBC3E55C94FF40E9F9
:101289000217B07F05D27F11171205FBC2AFC27FCB
:101299001117AE5CC3E55C947FD2AF500261331283
:1012A90005E7C2AF120625D2AFDFDA114EC3EE94BD
:1012B900057897F61206001217337F0AD27F1117A5
:1012C9001205FBC2AFC27F1117AE5CC3E55C947F08
:1012D900D2AF50E61205E7C2AF1206101205F1129D
:1012E9000610D2AFDFD6114EEE24037896F6F879C0
:1012F90097E7C394824003985006E824827897F6CA
:101309001206001216501217621205FB1117C3E5D7
:101319005C94FF5002414E0217B0757C00757D0048
:10132900C3E55C954C4003855C4C1205FB7801795B
:1013390088E7B403027805C3E55C984002412EC2F0
:10134900AF120625120625120625D2AF1206007520
:101359003000E4F531F5320531E531F4703F0532FD
:10136900789AE67819146012783214600D787D1431
:10137900600878FA146003753200C3E53298401D9D
:10138900120F0E1205E7153275310078998673C26E
:10139900AF120625D2AF789886731205FB1205F1B4
:1013A900E52A700530740221237801207402780639
:1013B900C3E55C9840A17888E6C3940360031205ED
:1013C900FBE52A7003021123C2AF120F0EE4F522C6
:1013D900F523F524F525F526F567D2AF7885E6C31B
:1013E90033F565E4F544F545F546F547F548F570F7
:1013F900F52CF52DF53775700875BB101205E71238
:1014090008A430EDFDA8BDA9BEE97001F8887112E4
:1014190008A875700875BB10120F8FC2AF7561FFF0
:1014290012091E852261852262852263D2AF752247
:1014390001752401752501752601856069756A01A3
:1014490075B69075A903757A017888E6B40307C261
:101459007D307602D27DD268D269753300120E676B
:0F146900120E9612093E12094512093E1209454C
:1014780012093E120BD3120706120CD4120D1B12BE
:101488000945120BC2306E031207072066031208C3
:101498005A30660312088A120CD4120D4A120945F2
:1014A800120BD3306E03120743120CD4120DC11263
:1014B8000945120BC2306E031207A1120CD4120D8B
:1014C800F0120945120BD3306E031207FE120CD42A
:1014D800120E671209451208A4120BC2120CD4127C
:1014E8000E961208A812094530692F856461856433
:1014F80062856069756A0179187A0CC3E533994089
:101508000CC269D26A8A357561FF021522C3E55C8F
:101518009401400302147B0215B0306A25206C2226
:10152800E535147006C26AD26B817BF535C3E55C7C
:101538009401400302147B7888E6C3940360030295
:1015480015B0753600788279A4E760027803C3E5A0
:101558005F985054307404E52A604D7888E6B403E7
:1015680017207D05207607A180307602A180206CA7
:1015780007D26C85646181BA78F0306C0585646146
:101588007820C3E541985002817B306C1BC26CC245
:101598007D307602D27DD26A753512856461817B91
:1015A8000536E55C6002A1B3753600C2AF120F0EB6
:1015B8007887E6FE7602120F8F7887EEF6E4F5223A
:1015C800F523F524F525F526F565752C00752D0010
:1015D80075A90075B680757A00D2AF1205FB120F97
:1015E8000E78A4E66006D295D297D293307409C3D8
:1015F800E536940440022123615B901A0D7820128D
:101608001692E520B45A0CA3121692E520B4A5034D
:10161800021630757CA5757DF1120F2312165075D0
:101628007C00757D0002164F901A0378807B0A12A1
:101638001692A308DBF9901A0F788C7B1912169270
:10164800A308DBF9901A2822C2AF1216D51216B2D7
:10165800901A00740E121697A37409121697A374A1
:1016680015121697901A0378807B0A121696A3080B
:10167800DBF9901A0F788C7B19121696A308DBF900
:101688001216E81216C6901A2822E493F622E643A8
:101698008F01538FFDFFC3E583941C400122EF8522
:1016A8007CB7857DB7F0538FFE22438F02438F01AD
:1016B800857CB7857DB7901A0DF0538FFC22901A60
:1016C8000D745AD197901A0E74A5D197227A307951
:1016D800D07820901A40D192E520F709A3DAF722B2
:1016E8007A3079D0901A40E7D19709A3DAF922AB7A
:1016F80074A875BB01027984BB02027985BB030219
:101708007986BB04027992BB05027987BB06027908
:10171800A3BB0702799CBB08027988BB09027989B7
:10172800E8F7227C05120600DCFB22C2AF12061085
:1017380012061712061E1206251205F112061012BD
:10174800061712061E1206251205F11206101206B9
:101758001712061E120625D2AF22C2AF1206251294
:10176800061E1206171206101205F1120625120699
:101778001E1206171206101205F112062512061E71
:10178800120617120610D2AF22AE74AF75C2AF128E
:1017980006101206101206101205F1DEF2120625C6
:1017A8001205F1DFF8D2AF22F133F12BF12B75746A
:1017B80001757501757600F1917C05AD5C12060026
:1017C800C3ED955C70F5C3E55C9401400AC3E55C24
:1017D80094FF40320217ECD1F7D150F133C2AF7504
:1017E800EF16F12BDCD50576C3E57694035002801D
:1017F800C6F12B0575E5741490009F93F808C3E5AE
:101808007598500280AE12172B12172B0574C3E57A
:1018180074940A5002809A120F23121650C2AF75A0
:05182800EF1612172B62
:0319FD0002107C59
:101A00000E0915FFFFFFFF03040A0301015AA50198
:101A1000FFFFFFFFFF03FFFFFF25D0FAFA04FF01DE
:091A2000007AFF0101000300FF40
:101A4000234656544C6962656532304150726F23AB
:101A500023424C48454C492346333930232020202B
:101A60002020202020202020202020202020202076
:101C0000C2AFC2D353D9BF7581C043B20343FF8073
:101C1000752438752503B1DC7529A5752AF175E29F
:101C20004043F12053A4DF75D4FFD2857DFA7803B9
:101C300079E67C10752200752300901DE97B0675FE
:101C400024987525013085028145208508D8FBD967
:101C5000F9DCF781B7308508D8FBD9F9DCF781B713
:101C6000B19CE493A3C39A6004DDC381B7DBDBB10D
:101C70008E6002812E7B08E493FAA3B16FDBF87AC1
:101C800030B16F752200752300B18EEAFCEBFDC305
:101C9000ED94FE400EB18E8A278B28ED30E0048A49
:101CA000828B83B18E7AC270D8C3ED94FE601950D6
:101CB000CEBD002BEC600F7520007521FF7529004B
:101CC000752A000200008100A827A9280809D80465
:101CD000D90281DCB192EA89AAF281CE0D81A3C337
:101CE000ED94035053EDA2E092007AC5C3E58294CF
:101CF00000E583941C508A200010438F02438F011B
:101D00008529B7852AB7F0300029A827A92808090E
:101D1000438F01538FFDD804D902A133C3E58394C7
:101D20001C4003A3A11689AAE28529B7852AB7F02A
:101D3000A3A116538FFC817F7AC1BD030CE493A34A
:101D4000FAB153DCF8B14B817F8181AA22AB23B178
:101D50006FEBFAEA6222752608C3E52313F523E543
:101D60002213F52250066323A0632201D526EAB18F
:101D7000DCB1DC75260AEAF4200102D285300102CA
:101D8000C285B1DCC3134002C201D526EB22B19259
:101D9000EAFB208502A192308502A197752608AE44
:101DA00024AF25C3EF13FFEE13FEB1E0B1DCC3EAAD
:101DB000133085024480FA30E703632201C3E52330
:101DC00013F523E52213F52250066323A0632201B5
:101DD000D526D9E52265236523F52222AE24AF2539
:101DE0000E0FDEFEDFFCD20122424C48656C6934E6
:071DF000373164F390060196
:00000001FF
